:20000000001C0020F1000000D1000000D7000000000000000000000000000000000000000B
:20002000000000000000000000000000DD0000000000000000000000E3000000E900000017
:20004000630100005D01000057010000510100004B01000045010000000000003F01000062
:2000600039010000330100002D01000027010000210100001B010000150100000F01000058
:2000800007010000FF00000000000000000000000000000000000000000000000000000059
:2000A000000000000000000000000000000000000000000000000000000000000000000040
:2000C00082001068116070478200106C116470472548806800472448C06800472248C06AC9
:2000E00000472148806B00471F48C06B0047704710B51E490020C86100F0E2FB10BD1A481D
:2001000080304068004718488030006800471648C06F00471448806F00471348406F0047CA
:200120001148006F00471048C06E00470E48806E00470D48406E00470B48006E00470A48B4
:20014000C06D00470848406D00470748006D00470548C06C00470448806C00470248406CAF
:2001600000470148006C004700100000401000F000000000000000000000000000000000EC
:2001800010B507E013469C00241F521E9B000C591B1FC450002AF5D110BD30B504460020B1
:2001A0000F221207136818258907AB43C90E0B431360116889088900491C1160411E2160DE
:2001C000116804231943116011684907FCD430BD10B500230F2212071468A408A400A41C6E
:2001E00014600160106804210843106010684007FCD4184610BDC849012008607047F0B522
:2002000004460020844620680F46401C1AD0C34E200A0502402231462846FFF7B1FF601BDD
:200220008010C117890F08188010800037500024A00031584019FFF7CBFF641C402CF7D3EB
:200240006046F0BD2046FFF7C3FFF9E7B44800210161B44A42618161B34A916003210161D7
:200260007047AF490020086148618861AE498860704710B500231A4603E0845CE3185BB20B
:20028000521C8A42F9D3D8B210BDA7488168491C81600120A54940064860704738B5A44A54
:2002A000010C1268012A06D10B221202914202D20122520789188B079B0FCA1A0004000E7E
:2002C00000259C4C6946102822D006DC012809D002280DD0042815D116E020281DD04028A8
:2002E00010D121E0104612680092227DCA5406E0104612680092A28A5B085B00CA52009916
:20030000FFF77DFF656138BD616910460091F7E710680090C85C207538BD58081268400051
:200320000092085AA08238BD1068606138BDF0B57F4A00241268010C012A06D10B22120228
:20034000914202D20122520789188A07920F8E1A0004050E0AE0A100764A88198F18796973
:20036000FFF74DFF00207861641CE4B2AC42F2D3F0BDF0B5704C87B020680590FFF771FFB1
:200380006D49601780310860634908606648012505616A490F20FFF793FE029068490020FD
:2003A000FFF792FE049067490120FFF78DFE0390FFF74CFF0121084600F0C8F82560022036
:2003C00020605C4800254562416A090A0902803141625D490020CA6B0092CA6B0192019B1F
:2003E000009A9A4207D1401C6428F4D94E4F3869002802D003E00020EDE7012A23D0B869AC
:20040000C0B24228B86947D0C0B25228B86946D0C0B2442846D044488069C0B25528D8D1A4
:20042000444F0026786A01210843796AC0B2090A09020143796234463D4920020968301847
:20044000012950D056E03A48056039494039C86901221043C861FFF704FF00203649C043CF
:20046000803108602C4908600F200299FFF728FE00200499FFF728FE01200399FFF724FEF2
:200480002D4905980860284805612A48416A090A0902416207B0F0BDFFF700FF21E0FFF7DD
:2004A00046FF1EE023480326416A760301221143426AC9B2120A12020A434262002420033B
:2004C000301A0121FFF769FE641C062CF7D31948416A426A0906490E4900120A12020A43F3
:2004E0004262BD6175E70B210902884202D20121490740180021FFF750FE641C102C9BD3B0
:20050000786A796A0006400E4000090A090201437962054885615CE780E200E0001C002051
:2005200000E000E0D5140000000C002000ED00E0401000F0001F002000E100E08B0200004C
:20054000F70100006D070000C06F0000F0B501231B04AE4A0029D16949D01943D1612024D2
:20056000AB4E102521030228F06942D08007C00FF7694000BF08BF000743F761A448403812
:20058000C6690F123E43C6619068FE26B04376309060106800090001C01C10601068204315
:2005A00010601068802420431060506828435060D0698843D061106A4C00A0431062106A3F
:2005C00008431062106A18431062106A000A00027630106238205063D069000A0002763083
:2005E000D0618C484168020291434160F0BD9943B4E7C007F369C00F9B089B000343F361E6
:20060000854803681B091B01DB1C0360036823430360036880242343036043682B43436040
:20062000036A8B430362D7E770B58407020AA40F12067A4B120E01D0012A03D105252D03C6
:2006400040195032764D1F2A32D0403A1F2A48D802462A40AD0652191568E400FF26A64092
:20066000B543A140294311606E4988420CD16E49CA680124E405A243CA60CA68A510AA438C
:20068000CA60CA68A243CA606849884229D1634A103A107C6649002444281CD00DDC1028AB
:2006A00012D0202813D0402813D0422818D112E002462A4001256D07CDE74F280ED05228CE
:2006C00009D055280CD106E00120086108E00C6106E0507C03E01868886101E00F2048616B
:2006E0001461002070BD010A10B50906090E01D0012903D105221203801850310B46103B82
:20070000474A0F2B04D8014611400122520713E00B467B3B742B05D80146114007221203D2
:20072000891A0AE070390A29014602D81140414A02E011400F221207891882070868920F9B
:200740003D490978CB073149CB6A07D0FF242402D200D040A3430006000C04E01B0A1B02F1
:20076000D200D040C0B20343CB6210BDF0B527490868FF22013210430860086810229043DC
:200780000860086B8006800E8863CA6A2A4C150C25608A6A120C62604B6A87069BB20126A5
:2007A0002361002F02DA5B192361A672C30603D523699B182361E672000700D5A672E07A90
:2007C000002500280AD0D007886A01D00004000E2072C1B22069FFF727FFE572A07A002803
:2007E00003D02069FFF77FFFA572144902200860F0BD09480168FF22013211430160026851
:2008000010218A4302600D4801607047009000F0401000F0004000F000A000F0101F00203C
:20082000FCFF00004E500000405000F0101F0000000C00200090FF1FE40C002080E200E044
:20084000000000000000000000000000000000000000000000000000000000000000000098
:20086000000000000000000000000000000000000000000000000000000000000000000078
:20088000000000000000000000000000000000000000000000000000000000000000000058
:2008A000000000000000000000000000000000000000000000000000000000000000000038
:2008C000FEB57D48426A02218A4342627B4C606B884360637A4882691204120E0A431102FD
:2008E0008269FF231B029A430A438261416980220902090E1143426909041B029A430A4300
:20090000426170480022C2616F49001708606F49086000F010F96E48026142610262426223
:2009200067486C491038002210234F1103E00A2A06D0092A0DD020C920C0052A14D018E085
:200940000D680095009D9D430095009D0126760204E00D680095009D0126F6053543009585
:20096000009D20C0091D04E0002500BF6D1CBD42FBD3521C102ADAD35748C169012212045F
:200980001143C161016809090901C91C0160016820229143016001688022114301604168CD
:2009A000994341608168FE22914356318160C169090A09027631C16161680122920511438D
:2009C0006160016A5211914301623B484030C16AC0229143C162C16A38221143C162C16A33
:2009E00006221143C1623D4C002020616061A061E061012525606060A060324E3068002880
:200A000046D0002000BF401CB842FBD32C48816982691943C9B2120A12020A43826100201D
:200A20002F49304E01273F0300BF401C8842FBD30020F16B0191F16B0291029A019991429D
:200A4000F6D1401C6428F4D9706B401C17D0B06B401C14D0706BB84210D9716B07200003DD
:200A600081420BD8716B3846091AFFF702FC1D492031097E08180006000E00D0256120690E
:200A8000012802D00198012813D0FFF772FCCFE700F036F80B480021403841631049B939A3
:200AA00081634104C1633560C1692943C1610020FEBD00F005FBBBE7005000F0004000F0BF
:200AC000405100F0401000F080E100E080E200E0001F0020187D0000009000F0000C002052
:200AE000B80B0000C06F000000000000000000000000000000000000000000000000000004
:200B0000012110B5002349070B200002401E1C5C0C54C028FAD801221203C020401E145C78
:200B20000B460C54FAD1084A0A600848084958608A62C86210BD07490020086148618861D6
:200B40000549486070470000001C0020F1000000001F002000E000E0000C00200000000090
:200B6000000000000000000000000000000000000000000000000000000000000000000075
:200B8000000000000000000000000000000000000000000000000000000000000000000055
:200BA000000000000000000000000000000000000000000000000000000000000000000035
:200BC000000000000000000000000000000000000000000000000000000000000000000015
:20100000001C0020F1000000411200004D12000000000000000000000000000000000000F1
:201020000000000000000000000000004F120000000000000000000051120000E9240000DF
:201040002D130000511B0000751B0000991B0000BD1B0000332E000000000000CB1200008A
:2010600095250000B1280000AD1200004D250000D5130000C1130000691300003113000030
:2010800057130000451300000000000000000000000000000000000000000000000000008E
:2010A000000000000000000000000000000000000000000000000000000000000000000030
:2010C000F8B501F01DFA0024524D01232B60524881680822114381608168042211438160C3
:2010E00081680222114381608168194381604B4900208200401C8C50C028FAD3484A0020B3
:20110000411E8300401CD1501028FAD301F0F9FE00207D21890100BF401C8842FBD301F097
:20112000D5FD01210846FFF711FA04F035FB0090684601788020014368460170009804F002
:2011400030FB0F2004F01BFB002003F0D0FF354804F0BDF80121802004F020F8012000F044
:2011600078FE012000F07EFE012004F036FB012004F047FB002004F0C1FA002004F0ADFA45
:201180000120800328608600304600F0BDFD304600F0CCFD301128600121022003F0D8FF77
:2011A00000F038FD20490869F2109043086102F039F901F0ADFF01F0B1FF01281BD0022852
:2011C00019D003281AD0042818D0032003F08FFF0321072003F0ABFFCF2003F04DFF022021
:2011E00003F07CFF0D4D803D02F063F802F051F8012806D007E002F0A7FEF3E703F068FA36
:20120000F0E703F0ACFD28690128EDD1044810380461F8BD00E100E0801000F0800C002048
:20122000101F002088130000005100F00348854604F0D0FC00480047C1080000001C002019
:2012400037488168C022914381607047FEE7704701203449C0064860704701203149400698
:2012600048607047FEE710B5112000F051F810BD10B5102000F04CF810BD10B50F2000F054
:2012800047F810BD10B50E2000F042F810BD10B50D2000F03DF810BD10B50C2000F038F863
:2012A00010BD10B50B2000F033F810BD10B50A2000F02EF810BD10B5092000F029F810BDEB
:2012C00010B5082000F024F810BD10B5072000F01FF810BD10B5052000F01AF810BD10B50A
:2012E000042000F015F810BD10B5032000F010F810BD10B5022000F00BF810BD10B50120C6
:2013000000F006F810BD10B5002000F001F810BDC106C90E01208840034908607047000085
:20132000801000F000ED00E080E200E07047000010B504F0F4F9032004F0E0F90F2000F0B2
:201340006FF810BD10B50021082004F0DBF9112000F066F810BD10B50021042004F0D2F96E
:20136000102000F05DF810BD10B504F0D8F91E21884344086400204604F0C0F9600603D596
:201380000121084602F03FF8200603D50121022002F039F8E00503D50121042002F033F82F
:2013A000A00503D50121082002F02DF8600503D50121102002F027F80E2000F031F810BD9B
:2013C00010B5FF200021013000F0A1FC0D2000F027F810BD10B500F0A6FCFF21044601314E
:2013E000884300F091FC204602F0A0FE204602F0BAFE204603F0CDF9600402D5012001F033
:20140000AEFFA00308D500F036FD012804D10848C169FF221143C1610C2000F001F810BD8B
:20142000C106C90E012088400249086070470000001000F080E200E010B5442831D014DC57
:201440002B283CD03C281DD040280DD103F0BCFE032803D004F072F9002803D0002001F080
:201460008BFF80B203F01EFF10BD462820D0482839D0FF385C28F7D101F0A9FF80B204F0BA
:20148000D8F810BD03F0A0FE032803D004F056F9002803D0022001F06FFF80B203F0FAFE44
:2014A00010BD012001F068FF80B203F002FF10BD032001F061FF80B203F002FF10BD01F09B
:2014C00028FF03F01BFF03F07FFE012807D0022805D0032805D0002003F019FF10BD012050
:2014E000FAE70220F8E700F0DAFB01467D20C00104F0CAF904F08DF810BD70B50025ED4329
:20150000F84E0C464E2807D0A02832D04F2844D1C8073ED001213DE0600601D5012000E037
:20152000002004F09FF8A00602D5012004F090F8E00603D50121042001F054FF200703D59F
:201540000121022001F04EFFE0071ED00121084601F048FF19E0A0071FD500F0B3FB012831
:2015600001D0012000E0002000F0A3FB0021062011E0600601D5012000E0002004F072F8F8
:20158000A00602D5012004F063F86007E3D5F561E1E70021082003F037FE70BD3EB5044646
:2015A00001F0B7FE002822D1022C20D100F081FB00200090694601900872684604F066F875
:2015C0000021022003F0D6FD0021802003F0D2FD0021022003F0BCFD0021802003F0B8FD27
:2015E0000021102004F07DF8002004F09CF83EBDF8B504460069BC4E010A87070D06BF0FAA
:20160000BA492D0E04D0012D27D01F2D59D027E082B24018502520613E2A1AD04E2A04D0F7
:201620004F2A0DD0692A1BD10FE0217A1046FFF764FF207A810713D5FD21084020720FE0AB
:20164000217A1046FFF759FF0AE0207AFFF7A6FF06E0022001F0E3FE02E040185125206121
:20166000403D1F2D44D8A24920690840890640180268F900FF238B409A43237A8B401343F7
:2016800003609A4920694E31884207D10021084603F0BAFD0021022003F0B6FD95492069F1
:2016A000884225D1904A103A107C93490023422818D00BDC10280ED020280FD0402816D1F6
:2016C0000EE08B49084001214907D0E74F280CD052280CD106E00120086108E00B6106E083
:2016E000507C03E03068886101E00F20486113610020F8BDF8B5064608690D46010A0906E1
:20170000090E01D0012903D1784A8018503128610A46103A76480F2A04D82969014001201E
:20172000400713E00A467B3A742A05D82969014007200003081A0AE070390A29296902D89E
:2017400001406E4802E001400F2000070818296904688F07BF0F65482030814206D100F030
:20176000B1FA01468020012910D08443FF2212022878002E0CD0C10761480029C16A0DD085
:201780009143FA00D4402206120C04E00443EDE7C1075C48F1E71143C162F8BD090A090294
:2017A000FA00D440E2B2F6E7F8B5FF220132554F0026054600280ED05148534C8169036801
:2017C0008907C90F13430360026810239A430260002923D023E04C4CB869A41F8007396849
:2017E000C00F114339603968102291433960002800D1667078684006C00FA07030D000F029
:2018000020FA012805D1F868E178000A00020843F860386902210843386109E06670416837
:201820004906C90FA17008D00169022211430161A07800281BD1002D12D03148C069000473
:20184000070E607800280DD001280DD002280FD003280CD16079002860D0012874D193E06D
:20186000F869ECE7012001E0677102206070F8BD2771A088FFF7E0FD002D2AD100F0E1F92E
:20188000012826D160790011801F030004F0B4F909060B0B0B0B0B0B0B0B1100A188012039
:2018A0004007081802E0A088184940180078E0700FE0A08881080F2089000007081821791D
:2018C0008907890F08D0012908D0022920D0032921D06078401CC9E70068E8E70068000447
:2018E0001AE00000001000F0101F002000500000FCFF0000101F0000000C00200090FF1F4B
:2019000000A000F0009000F0860C00200090FFFF0068000200E00068000EC8E7A08850216F
:2019200061712179672901D16D212171002D04D0692825D0A02832D119E04E2805D04F28AC
:201940000CD069282BD10EE020E039464E20FFF7D4FDB8071CD5FD20074019E039464F2081
:20196000FFF7CBFD14E03846FFF718FE10E03946A020FFF7C2FDB80711D5FD2007400EE050
:201980003846FFF70BFE0AE051206071002D06D160791F2809D006280ED007280CD0A08862
:2019A000810889000F20000704E0A0888108890001204007081806E0A088FF21FD31084095
:2019C00001214907401821798907890F06D0012909D002291CD003290CD11FE00168090A07
:2019E0000902394305E00168FF22120291433A0218E00160A088002D16D07D49884203D1D5
:201A00000021084603F09DFDA088401CA080F8BD0168FF22120491433A0403E00168090268
:201A2000090A3A061143E4E771495239884207D10021084603F0E8FB0021022003F0E4FBF3
:201A4000A0886C498842DFD16B4A6B4B103A107C6A49402817D004DC102807D0202819D1CB
:201A60000FE0422811D04F2814D111E0012008616349886AFF231B029843FF300130886253
:201A800008E00E6106E0507C03E01868886101E00F204861166110690090B5E7F8B5594EC8
:201AA000594F05002FD0594C386B8006800EB863F96A090C2160B96A090C6160796A8206A6
:201AC00089B221610121002A04DA23682269D2182261A172C20604D563682269D218226125
:201AE000E172000703D5A1722069FFF7A5FCE07A002821D02079C00715D0002D11D0B86A99
:201B00000004000E12E0414C306B143C8006800EB063F16A090C2160B16A090C6160716A65
:201B2000CDE7B06AECE7002D10D0B86A20722046FFF75EFD0020E072A07A002805D021469C
:201B40002846FFF7D7FD0020A072F8BDB06AEDE710B52C480168FF22013211430160016864
:201B60001022914301600020FFF798FF012000F037F810BD10B524480168FF220132114302
:201B8000016001681022914301600120FFF786FF022000F025F810BD10B51A480168FF22CB
:201BA00001321143016001681022914301600020FFF7FAFD032000F013F810BD10B5114857
:201BC0000168FF2201321143016001681022914301600120FFF7E8FD042000F001F810BDED
:201BE000C106C90E012088400949086070470000A0500000101F0000101F0020000C002053
:201C0000405000F0009000F000A000F00C0D002080E200E0FE49002008707047FD4A516B20
:201C20000223C0079943800F014351637047F94A51680123DB03C0079943000C01435160FC
:201C40007047F44800680006C00F7047C907F14AC90F0028506805D053029843C9050843BC
:201C60005060704701239B0598438905F7E710B5E8480069E84C01052078090D49304843A8
:201C8000C82103F001FEE54980B24843E44903F011FE01216156C900401880B210BDDD4831
:201CA000006AC004000D7047DA48006AC000C00C7047D84A516B8023C0079943000E0143ED
:201CC00051637047D348406B0006C00F704710B5D04CE269D34B9202920A1A400303134317
:201CE00088051843E06110BDCA4AD169CC4B5B42194040000843D0617047C64AD169490885
:201D000049000143D1617047C24908637047C14A012905D0002902D1116B814311637047AF
:201D2000116B0143FAE7BB48806A7047B949C8627047B84A012905D0002902D1D16A81437F
:201D4000D1627047D16A0143FAE7B24A11689301C0079943C00A014311607047AD494A68AF
:201D600003781202120A1B061A434A604A6803239B049A4343789B071B0B1A434A604A6800
:201D800003231B049A4383789B079B0B1A434A60A04940310A68C378120912011B071B0F56
:201DA0001A430A600A680079F02300079A43000E02430A607047012805D002280DD00428D5
:201DC0000DD008280DD00020924A516803235B03994340030143516070470120F4E70220F7
:201DE000F2E70320F0E78B494A6807239B029A4303785B07DB0C1A434A604A687C239A43ED
:201E00004378DB065B0E1A434A604A68FF2301339A438378DB07DB0D1A434A604A68C0781B
:201E20008023C0079A43000E02434A60486B4022104348637047774A51687C23C0069943D9
:201E4000400E014351607047724840684006C00E7047704A516B1023C0079943C00E0143FD
:201E6000516370476B4A516B0823C0079943000F0143516370476748406B400301D5012066
:201E80007047002070476349496A014201D001207047002070471CB55E49CA686B46120E17
:201EA0001A70CA681202120E5A70CA681204120E9A70CA681206520FDA70C9680522C906DA
:201EC000C90E1971194603F009FD1CBD51490068886070474F480830006870474D490068E3
:201EE000086070474B4800687047F0B5494C85B0010011D001292BD0022974D0032809D127
:201F0000606949490001000D4843484903F0D2FC4749401805B0F0BD012102A800F0A6FFD0
:201F2000039902980191009020696A4601051078090D49304843C82103F0BCFC37494843C9
:201F4000374903F0B7FC6A465188C90009B2E0E7206900210001040D02A800F087FF03990F
:201F600002980191009000F07EFF012811D003F02BF903280DD04127FF00FF25E135244802
:201F80002C4E0078002809D003F008FB012819D01DE0FF274137FF251935F0E76A46107929
:201FA000C8214930604303F085FC23494843234903F080FC6A460621515E40181449012278
:201FC0000A7043E07069B84201D9002007E003F0E5FA002808D17069A84205D2012003F02F
:201FE000EFFA706932E046E003F0D8FA012803D100F039FF00282ED06A461078C82149303D
:20200000604303F057FC0C494843054918E000008C0C0020004000F09F0C0020E880000096
:20202000FF0F0000FF0FC0FF74B90200102700005C95FFFF200D002098080000FD2F000057
:2020400003F038FC6A460221515E4018002800DA002070615EE76A461079C8214930604309
:2020600003F028FCE2494843E24903F023FC6A460621515EE9E7606901210405240D02A831
:2020800000F0F4FE039902986A46019100901079C8214930604303F00DFCD7494843D74901
:2020A00003F008FC6A460621515EC90040180028D0DC00202EE7D24800210160416081605B
:2020C000C160016181617047CE49486AC005FCD5CB480B6902681B051B0DD2180260426856
:2020E0000B691B011B0DD218426082684B691B051B0DD2188260C26849690901090D511885
:20210000C1608169491C81617047BE48416AC905FCD5BB4903694A681B011B0DD2184A606C
:202120000A6980690005000D101808618869401C88617047F0B5B24C85B0A169030003F0DB
:202140005BFD0504219ABBC6B900012102A800F08DFE0399029801910090A169206803F005
:2021600093FB6A461278C8214932504303F0A2FBA1494843A14903F09DFB6A460221515EA4
:20218000C900A2E0002102A800F070FE0399029801910090A169606803F076FB054600F002
:2021A00062FE012810D003F00FF803280CD04127FF00FF26E13694480078002809D003F0CA
:2021C000EDF9012819D01DE0FF274137FF261936F1E76A461079C8214930684303F06AFB82
:2021E00083494843834903F065FB6A460621515E4018854901220A7028E06069B84201D97B
:20220000002007E003F0CAF9002807D16069B04204D2012003F0D4F9606917E003F0BEF925
:20222000012803D100F01FFE002814D06A461078C8214930684303F03DFB6D4948436F491F
:2022400003F038FB6A460221515E4018002800DA002060615EE66A461079C8214930684311
:2022600003F028FB62494843624903F023FB6A460621515EE9E7012102A800F0F7FD0399B4
:20228000029801910090A169A06803F0FDFA6A46117949314843C82103F00CFB564948433A
:2022A000564903F007FB6A460621515EC90040180028CFDC00202DE6E06803F0E5FA534927
:2022C0004843534903F0F6FA5249401822E6206903F0DAFA1EE670B50D464B494A68824223
:2022E00026D0486001464C4803F0E4FAC41EE00700D1641C7D22D200511B20464843114655
:2023000003F0D8FAC10700D1401C3E498A6B434B1A40E3055B0D1A438A638A6B404BC005C0
:202320001A40000B02438A63886B02221043886370BD10B50146384803F0BCFAC41EE00786
:2023400000D1641CFF212046F5314843490003F0B1FAC10700D1401C2A498A6B2F4B1A40DD
:20236000E3055B0D1A438A638A6B2D4BC0051A40000B02438A63886B02221043886310BDD8
:20238000284910B5091A642041431F484160224803F090FAC41EE00700D1641CFF2120464D
:2023A000F5314843490003F085FAC10700D1401C14498A6B194B1A40E3055B0D1A438A6312
:2023C0008A6B174BC0051A40000B02438A63886B02221043886310BD0B4840687047094924
:2023E0008A6BC00752085200C00F02438A63704798080000FD2F0000E8800000FF0F00007B
:20240000200D0020004000F08C0C002074B90200102700005C95FFFF0048E80103F8FFFF08
:20242000FF07F0FF6C0700002C48012141740021C17470472948C07C7047F8B5274C607C7C
:2024400000281ED0002565740120E074FFF7C4FF014620607D2000010E18214F66603846FB
:2024600003F012FAA0603146384603F00DFAE06025740220A0747D20400100F097F800F012
:20248000A1F8F8BD70B5154C0025207C422806D300F09EF8FFF7A0FFFFF74BFFE574207C14
:2024A0001049085C01280DD0A06800F097F8A07C002802D02068FFF73CFFA574207C401CF2
:2024C000207470BDE06800F089F8A07C012802D06068FFF72EFF0120A074EFE73C0D00200C
:2024E0000040420F305C000023480168491C0160012022494006486070471F48006870476E
:202500001F48002101611F4A426181610321016170471B4800210161416181617047164926
:202520000A680B689B1A8342FBD9704716480268012109038A4302607D221201C261134B59
:202540004A101A6002680A43026070470A484168491C41600C48416A0822114341620C4961
:2025600010020860704704484068704710B57D2103F08AF910BD0000940C002000ED00E04C
:2025800000E000E0D514000000D000F000E100E080E200E010B5FE48416A012211434162FF
:2025A000FC4910020860FFF76DFF10BDF8490A68520852000A6000014860FF20F64901302C
:2025C00008607047F24801680122114301607047EF4801684908490001607047EC49000122
:2025E00048607047EA480168C9062DD40168102211430160E948018B491C0183018C028804
:20260000891A8186018B0E2907D8028C018B49000918FF31FF3102318A873421415E002929
:2026200001DD012101E00021C943DD4A1171418B00224B00C9180918C0314A75418B4B00E1
:20264000C9180818C0300275704710B5D0480168102291430160D2490020087602F07CFB8C
:20266000032809D1CE482030007F002804D1CD48016849004908016010BD10B5C748008BCE
:20268000C949884207D2FFF738FFC5492031C968401A642804D9FFF7D8FFC1490120087491
:2026A00010BDF8B50D46BE49097E002922D0BB4F012D398807D0081804B2FFF7DEFF052006
:2026C000C0013E1819E0081AF6E7B848016BFF22013211430163416AC905FCD5806900053B
:2026E000000D3884B248012D385E04D0A04204DCFFF778FFF8BDA042FADCFFF7FEFE716818
:20270000401A0128E1D9F8BDF8B5FFF79EFFA44D01202874E87C002816D12F462037B8786A
:20272000002811D100249D4E06E030194030007A02F064F8641CA4B2A87CA042F5D8706898
:202740003080FFF7DAFE3862F8BD30B5934B4033187A010992488174827C01462039002A43
:2027600017D0827C921C8274827C0B246243CA858B4A002420329470847C0A2C02D21B7AC1
:20278000002B05D1042383742C20C8850120907030BD032282742122E9E7804B10B5591844
:2027A0004031002808D0421E072A07D8087A5C8B5C33E35C93401843087210BD0928FCD18E
:2027C0007748C27C097A4A40C27410BD70B57448007D01281BD1714C608B0B2103F054F866
:2027E000608B0D460B2103F04FF8C1B22846FFF7D4FF608B401C6083608B0B2808D0608B80
:2028000067492039C98D884201D1FFF77DFF70BDFFF79BFF70BD5E480168102291430160EB
:202820007047F8B500225E4E1346203EF18E104600293CD1594C02214D002D19FF35FF35E1
:202840000235AF8F6D8F7D1B2DB2322D05DD01280CD05B1CDBB2012008E03227FD4205DAC6
:20286000451C03D0521C0020D2B2C043491CC9B20E29E1D90125022B03D3022A01D3F5869A
:2028800011E0FFF7E2FE4648057402F065FA032809D143482030007F002804D141480168CB
:2028A0004900490801604348208200206082F8BDF8B53748416A02221143416201253549A3
:2028C00010020860354F388B401C3883388B052102F0DAFF0E46FFF7D0FE3448016B2A0240
:2028E00011430163416AC905FCD5806972000105090D384614182184218C3A88891AA186D7
:202900003422A25E0021C943002A01DD012300E00B46132287195201BA181371204F3B7D32
:20292000002B0CD02022A25E1423C35E9A420BDC428B5300D2181218C032517510E0042330
:20294000D356002B06DCF3E72021615E1622825E914205DB418B4A0089180918C0310D7551
:20296000018B00290AD0018B0E2907D8218C028B52001218FF32FF32023291870748008BE8
:202980000E2801D1FFF74DFF0448008B282813E000D000F080E200E000E100E0500D002093
:2029A000B00F0020801000F002030000004000F020000000FF7F000028D3BD48018B302900
:2029C00024D81021415E2022A25E914202DD218C018207E01221415E2022A25E914201DA5E
:2029E000218C4182018B302910D104461220205E1021615E401A142102F05CFFC1004018C2
:202A0000218A0918A182618A081AE082042E4BD1A74B2820185E1421595E884207DC588BDE
:202A2000002142008018C018C03081750BE02820185E1621595E884205DB588B4100401820
:202A4000C018C0308575FFF7E6FE188B994C1D2802D81D26F64320E0188B312801D80026BC
:202A60001BE01026A65F217A588B42008018C018D62282568E485C30914202D0598B0D54D4
:202A800009E0397D002900D13D755A8B00211154207A68402072FFF799FEFFF72EFD60603E
:202AA000217A3046FFF7FDFDF8BD83490A6810239A430A600001C86080495801086070473E
:202AC00010B57D480168C90630D4016810221143016002F041F9032804D179480168020682
:202AE00011430160FFF709FD7249C860704800210183028C0388D21A82863422825E002A78
:202B000001DD012301E00023DB436A4A203A13716C4B038241821346203BD9860123137640
:202B200041836348403003770172D17410BDF8B5FFF7E3FC05465E4E0020F060B060FF2798
:202B4000614C01370EE0206B38432063606AC005FCD5B068A1690905090D4018B060F068B3
:202B6000401CF060FFF7C9FC401B0228EBD9F168B06802F089FE30800020305E70603088D5
:202B80003084F8BD4B4910B501202039087448480024048344830C7504228A74454A2D21F9
:202BA000403AD1854749018244820188C183FFF7A4FC4049C8600C77FFF747FD10BDF8B521
:202BC000064602F00AF90446FFF797FCFFF795FC001B0A285BD3FFF72DFC012857D002F07E
:202BE000F9F8012853D0334C203C207E304FFD1DFF35FA35002837D13348016BFF220132B8
:202C000011430163416AC905FCD580690005000D3884388C3988401A694608802548012156
:202C20000172694600228A5E002A05DA0A460988494211800021017269460988891B018069
:202C4000398C4182068269460020085EB0420BDDFFF753FCE96F401A022802D9FFF730FF34
:202C600002E0FFF74AFCE867207C01280FD1002020743883788320750420A0740D492D2068
:202C80004039C88538883884FFF737FCE867F8BD08482038007E70470549486070470548EE
:202CA000C06870470349087770470248006A7047500D0020D00F002000D000F000E100E04B
:202CC000801000F0FF7F0000004000F0F8B5032034494002C8613448016809090901C91C28
:202CE0000160016820263143016001688027394301608168FE2291437631816041681022C2
:202D000011434160C16914032143C161C169090A09027631C161C1695503A943C161026AEA
:202D2000A1008A430262016A29430162016A2143016200210846FEF789FF1C48016809098A
:202D40000901C91C01600168314301600168394301608168FE22914376318160416810225F
:202D600011434160C1692143C161C169090A09027631C161C169A943C161026AA1008A438B
:202D80000262016A29430162016A2143016200210120FEF75BFF064802210160042101607A
:202DA000F8BD0000001000F0009000F000A000F000E100E026498A699206FCD40A68120A35
:202DC000120202430A60704700B5034602E05B1CFFF7F0FF18780028F9D100BD10B5012315
:202DE0001C48202101601C48C3631948826B0A438263416A090C0904891C4162816A090CAE
:202E000009040B318162016B1A0211430163104940318A68022422438A60C16A1022114364
:202E2000C162C16A60221143C162016B1943016310BD0A482021016005484030026892069F
:202E400002D542680A43426001684906FCD4704700B000F000E100E0401000F080E200E0E0
:202E60009F49887070479E48807870477CB50C46054602F0A9F903280FD0002C16D0012C7B
:202E800030D000216846017041800171C18008226946284602F022FD7CBD91496A461C3116
:202EA0000878107048885080081F0CE08C48807801280DD08A486A46143001781170408805
:202EC000508087481030017811714088D080DEE783486A460C30017811704088508080482A
:202EE0000830F0E77E486A46C01C01781170012141565180801C0178117101214156D1804C
:202F0000C5E7FCB57D221202126876A179A0552A7ED17B4B7B4A002403E00A2C79D0092CE3
:202F200078D015681D6001256D02AE03641C121D1B1DE4B2102CF0D3694A724B921C3C3300
:202F40001B7813706F4B521C3E331B7813706D4B3F331B7853706B4B921C40331B7813703F
:202F6000684B41331B785370664B133242331B781370644B183A43331B781370614B521CAC
:202F800044331B781370531E5A781C78120222431C4618346280221D5A4C45342478147046
:202FA000584C1C3A463424781470564C521C4734247814705A781C78120222431C461C3441
:202FC00062804F4A1032146A2404240E2502146AE4B225431C4610346580156A166A2D0EF4
:202FE0002D023602360E3543261D7580556A566A2D042D0E2D02F6B235431E4608367580A5
:20300000556A2D0E2E02556A2D022D0E2E4302E064E015E019E0251F6E80966A2670966A10
:203020003604370E261D3770966A3602370E2E1F3770926A120E2A709A78FF2A0DD021E0E7
:2030400017680097009F2F4303E017680097009F37430097009F1F6068E700229A70204E99
:2030600062801436374672800C3F7A806A807F23237033703B702B707C1F23706270A41CA8
:2030800023706270214B204A5A601D4A803A00239C000D5D6418E67836063543A678647869
:2030A0003604240226433543019520C25B1CDBB2032BEDD302CA00218B00C45C1B18DD7845
:2030C0002D062C439D785B782D041B021D432C43019410C2491CC9B20229EDD3FCBD00005E
:2030E0009C0C00204175672031362032303138200000000032333A32393A353600000000AA
:20310000305100F0187D000000000410005000F0C64800210170C17701777047F0B5002089
:2031200085B07D240546E4000646039002F04CF8012701287ED002287CD003287AD00820C3
:20314000FEF739FE002001F0D2FFFEF7CBFE40210843049004A8FEF7C1FE19214901481027
:20316000FEF7B5FD0520FEF7BFFD0020FEF7C5FD01218803FEF7CBFD01218803FEF7D9FD19
:20318000AB4938030860FFF7B8F90746FFF7B5F9C01B052803D8FEF782FD0028F6D0A349CF
:2031A000002048700120FEF742FDFEF778FDC008A84200D90546A04200D204460399761C76
:2031C00008180390FFF799F9C01B0528EDD93146039802F059FB954E2A1B03217060042A44
:2031E00003D9641F3C2C04D922E002464A3A682A02D2012030700FE0102819D8707801280D
:2032000016D000203070B0770121202001F0A0FF0121102002F0D1FA7D20C001716802F0B7
:2032200033FB02F0FEF90020FEF701FD2DE001E03170F1E70120FEF7F1FC0020FEF739FDAF
:203240000021022001F096FF0021802001F092FF0021022001F07CFF0021802001F078FF8A
:203260000021102002F03DFA0024009468460194047202F00BFA0021102002F09EFA012070
:2032800002F0FAF96948877704706848007805B0F0BD10B501F098FF032801D0002010BD66
:2032A0000021102002F089FA012002F0E5F9012010BD38B501F088FF5C4C012810D0022829
:2032C0000ED000280BD1A07F012808D10121102002F073FA012002F0CFF90220A07738BD31
:2032E000A07F0028FBD10120FEF798FC002020700098C008C00000906846FEF7EFFD012001
:20330000A0770021102002F058FA012002F0B4F938BD464800787047444908707047434848
:2033200040686338152801D801207047002070473E484068642801D3012070470020704748
:203340003A48406801464B39172901D8012070476338152801D802207047002070473349AA
:2033600048707047314902688A604268CA6082680A61C0684861704710B52C490A78012A78
:203380000AD0022A08D0002819D0012817D0022814D0032808D112E0002807D0012807D02B
:2033A000022807D003280DD0002010BD886810BDC86810BD08691F498842FADA0220FEF7CF
:2033C00094FD10BD486910BD1849886170471748806970471549097F014201D0012070473F
:2033E00000207047114B01291A7F02D082431A7770470243FBE70D49497F014201D001207E
:20340000704700207047094B01295A7F02D082435A7770470243FBE70448C07F70470349F3
:20342000C87770470149002088777047F40F002000E100E0B80B0000F8B5054616460F4626
:203440000120FEF7F8FCFEF712FC84091F20FEF7F2FCFF2C00D3FF24FC48446001202870EE
:203460006C701E203860072030607120F8BD70B50446022015460E46207001F059FF6070B4
:20348000C820306000202860012070BD38B50400EF48F04A09D0012C0ED0FF221E32022CD9
:2034A00011D05F2916DA00241FE081421CDC914218DCBE2910DC18E05F29F4DB814213DC3A
:2034C00091420FDC11E05F29EDDB914204DB81420ADC0AE0914201DA012406E0FF20C330DD
:2034E000814201DA022400E0032402F055F900906846C321BF220078002C0ED0C30708D09A
:20350000084040084000104069460870009802F048F9CE480477204638BDC307F9D10840D1
:203520000121001D0843EEE7014610B5C7480129C07E09D1410601D5801C04E0002806D034
:20354000012806D0801EC0B202F05AF810BD4120FAE74020F8E770B5BF4C002521780122B9
:203560002E46002904D0012906D002290ED019E06E280FDC002010E0B649884202DD02207D
:20358000607009E0322807DA6670F3E7FF211E31884201DA62700BE0032001F0B1FD20785C
:2035A000002805D06078002802D1A078401CA070A078002807D0401C7D25C0B2ED00A07033
:2035C0000A2800D3A67060782070284670BDF7B50D469E490646887F88B0782801D2401C8D
:2035E00088779A48C07C002832D00020FEF7A2FD04460120FEF79EFD04900220FEF79AFD93
:2036000007460320FEF796FD0590FEF754FD0498009401900598039002976846FFF7A2FE09
:20362000FEF76BFF89498D4F8968401AB84203D88948C078002819D0FEF75FFF8349896833
:20364000401AB84272D9844FF878002867D089E0322028607D483724817F0327032902D39B
:203660000121C17428270021417771E1774FB87F08281BD07A48844202DD387D022805D046
:203680007848844225DD387D022822D0387C032834D00120FEF70DFB012002F044F80A2057
:2036A000FEF73DFF6C490120C87027E07868A04201DD01200BE07D204001844201DD022074
:2036C00005E06948694920188842F2D90020387514E0FEF712FFB968401A7D210901884221
:2036E0000CD9387D022809D00020FEF7E2FA002002F019F800205E49C043C8615948001B6A
:2037000000B2C117C90E081844117F2C01DD7F24BBE07F20C043844200DA0446B5E04B4858
:20372000007D022803D0012803D011E01CE0514800E04B4884420BDD0120FEF7BAFA012081
:2037400001F0F1FF0A20FEF7EAFE0120F87009E00020FEF7AEFA002001F0E5FF00204449B0
:20376000C043C861012038713B4F04997879FFF78DFE7871032817D00020FFF771FB00201D
:20378000FFF7D2FE34484079002812D0012813D0022814D02820069001F0A8FD07B2354860
:2037A00087420EDC05210DE00120FFF759FB0120E6E74B200001EEE7AF208000EBE7C820A0
:2037C000E9E70A2121480170007C032819D00498FFF7C1FE059001F085FE1C49097C062911
:2037E00014D02548381887B23846FFF7EDFD0498322811DA381B00B2C117490E0818C41187
:2038000010E0002001F07CFC0020E3E706997918091805980818E6E7381B00B2C117C90EB6
:2038200008184411322C01DD322404E03120C043844200DA044608484079002801D0012834
:2038400023D1A01E302819D8641E1EE0141000208A0200007C010000BC0C0020881300001D
:20386000641900004C1D000047F4FFFFE7030000001000F07C150000C40900002046323019
:20388000312801D2641C00E00024F948007C032802D1F84900208871F6480B21807901F00F
:2038A000F3FF0A2922D0307851280ED00420FFF791FD01281CD00120FFF78CFD01281FD07D
:2038C0000220FFF787FD012822D00327FFF7A4FD8021012826D0E74802793720002A03D0B2
:2038E000052C01DA621D1DDC28601CE00427EDE7052700210420FFF775FD002103200EE0B6
:20390000282700210120FFF76DFD0021072006E0022700213846FFF765FD0021042001F032
:2039200073FCD3E729600A99002008603078282804D0032805D0282803D009E070780C28B6
:2039400003D0CB48007C032802D10120FEF773FA03203070C74974708879421C8A710B2840
:2039600001D10020887138460BB0F0BDF7B588B00020FEF7DFFB06460120FEF7DBFB054620
:203980000220FEF7D7FB04460320FEF7D3FB0746FEF791FB02A80597029603950494FFF73C
:2039A000E1FCB34C1C202178205601AB6A4601F02AFD6846007802F098F807466846007950
:2039C00002F093F805210690C943384602F076F87F21C90501F09EFF0746A749069801F0FC
:2039E000F2FFA64901F096FF0690207802F07DF80790284602F06EF8A14D294602F020F808
:203A00000446304602F066F8294602F019F8394601F0D9FF214601F0D6FF069901F07AFFA6
:203A2000072102F04BF8079902F00AF802F064F800B2FF2801DDFF2002E0002800DA00206D
:203A4000089904220A700899487009987D2101600A9800210160032086E770B504460520E4
:203A600015460E46207001F05DFC6070C820306000202860032070BD0623037064234370A7
:203A800032200860002010605120704707230370AA23437000200B6010601846704709235B
:203AA000037000234370AA2008601360704710B52023037043780024002B0CD0012B0CD0F8
:203AC000022B0DD0032B0DD04470AA2383700B601846146010BD012300E002234370F4E79C
:203AE0000323FBE70423F9E722230370AA234370837000200B60106018467047F7B55C4F25
:203B000004460E46787F0522022182B0002811D1B87F03280ED32820207006206070A27067
:203B2000787F002803D02825401C78771DE0F9740325F9E7387C012823D0042821D06846EE
:203B400001F0FBFB68460078207068464078607068468078A0706846C078E070684600797F
:203B600020716846407960710325462030606078401F030002F040F80826202626262626EE
:203B8000102618202070FF206070B87C012801D03974E9E73A74E7E7387C022801D0062834
:203BA00007D10020387678767875032038740120B8748020306005E0A0782C2802D10120F3
:203BC000FFF72DFC049900200860284605B0F0BD31230370AA238370C37046200860002029
:203BE00010603120704710B5512303700A23437000238370C37082240471437146200860DB
:203C000001201360FEF725F9032010BD54230370AA2343708370C370037143714620086087
:203C2000002010601846704755230370AA2343708370C370037143714620086000201060C8
:203C4000184670477123037011234370002383704223C37064230371B723437135238371DE
:203C60008A23C371432351200B6007211160704714100020BC0C00208FC2753C3333F3BF8B
:203C800000007A4481230370002343708370C370037143718371C37103724320086006209D
:203CA0001360E4E7F0B5FB4C89B005262670002020746074A074E074E07560762076A07619
:203CC0006077A0772146E077203108702075FFF7A6FB0F2701253846FEF716F83846FEF7F3
:203CE00025F8ED4928030860FEF7FCF8C008C000A904401C0843079007A8FEF7EFF80D20CA
:203D00006A4610700220507095700820D07010716846FEF723F803206A4610761F20507687
:203D20009576D57606A8FEF75EF8C32001F0A4F9022001F0D3F96A46167396205073967329
:203D4000D0730B2010748A2151749074D174162010757A205075142090759920D07503A8BC
:203D600001F000FBCD4801F03DFA012001F028FCC02001F039FC002001F0C2F903210720C7
:203D800001F0D5F90120FDF749FF01F0AFFAFFF71BFB0020FFF764F801F02EFCE07601F08D
:203DA0005BFD6A46107AC321084010302843BF2108401072029801F0F4FC09B0F0BDF8B562
:203DC000B44F0546387C3C4644340026030001F013FF0604B2B23CB2A8B20220FEF79FFB54
:203DE0000120FDF7B2FFAB48417D491C4175FEF784FB07460AE0FEF780FBC01B502805D3EB
:203E0000207A002807D0E07901280BD0FEF775FBC01BC828EFD99F48417D032940D30221AD
:203E2000017473E09B482430017F0229F3D1407F012806D00028EED1964801214674017440
:203E40005BE0944801214174F9E70220FEF767FB0120FDF77AFF8F48417D491C4175FEF7E8
:203E60004CFB07460AE0FEF748FBC01BA02805D3207A002807D0E079012815D0FEF73DFBE4
:203E8000C01BC828EFD98349487D032808D3487C012842D0002840D08E74062008744E755A
:203EA0000020FDF752FF4AE0207A022816D379482430017F022911D1407F012802D0002842
:203EC00007D00BE0734801214174017E491C017604E070484674417E491C41766D48017ECE
:203EE000022904D3042101740121417405E0417E022905D304210174467446752825CFE796
:203F0000417D032906D3417C012901D04675C7E7042194E703210174C2E7042008742825EE
:203F2000BDE7797C0022022001F07CFC0620BE743874032506E0FDF787FF1F2802D01F2057
:203F4000FDF779FF2846F8BD1FB5FFF7ABFEFEF7D4FA50498860FDF7C5FF0190FDF7BAFF25
:203F60000090FEF7CAFA0446FEF7C7FA001B022805D8FF200130FDF786FF0128F4D11420EB
:203F8000FEF7CDFA0124FEF7B8FA45480021CA00825CA24209D1C900081843683D4803AABF
:203FA00002A924309847044603E0491C89B21129EDD3384D24352978202901D2012019E0A7
:203FC000802907D208462038C217120F10180011801C0FE0E029084606D28038C217520FDA
:203FE0001018C010083005E0E038C217920F101880101430C7B227486F752530A863A975D4
:20400000002007E0AA6BAB7D1678521C7340AB75401CAA638742F5DC1E4800262730A8639C
:20402000EE752E761930E863001DC67106726A46117068785070A8789070A87DD070684615
:20404000FDF744FF1F20019940028143687DC006800C0143FF200130014301A80191FDF70C
:204060003DFFFEF74AFA0746FEF747FAC01BC82802D8287E0128F7D12E76FEF73EFA0646EF
:204080002878022816D0032817D005280AD0282822D10AE01410002000E100E09A99993F1A
:2040A000745C00000021032001E00021072001F0ABF811E000210420F9E72046FFF77FFE40
:2040C0000446FEF71AFA0299C01B884204D9FEF714FAC01B001D02900398FEF720FAFF2515
:2040E00001350EE0032C01D0042C0AD1FEF705FA801B152805D901212846FDF708FEFDF769
:20410000E3FFFEF7FAF90299C01B8842EAD90120FFF760F9012800D035E728240021FFF7EA
:2041200061F90021072001F06FF82CE738B50446FDF7D0FE00903A49E00701D0012008760F
:20414000A0070FD5C87D6B46401CC875C007886B027801D05A7000E09A70401C88631846E7
:20416000FDF7B4FE38BD1FB5044602A8FDF793FE0399019102982A490090600720310028AC
:2041800040DA68460079264B002809D01D282CD0487A0A7A401C824268462AD1007829E09B
:2041A00068468278D86B0270D86B401CD863202A01D2012217E0802A06D2203AD017000FBF
:2041C00080180211921C0EE0E02A06D2803AD017400F8018C210083205E0E03AD017800FAD
:2041E0008018821014324A7209E068468078487105E04078DA6B1070D86B401CD863087A8D
:20420000401C0872200708D56846C078002805D000228A7188720120C8711FBD0122F8E792
:204220003810002070B50646FF480D460721036849068B43012109060B4314460360FDF72B
:204240004DFE002030742060F8482860022070BD70B5F54B0D4606460721186849068843F2
:20426000032149064018186014461846FDF736FE0020307420607D2000012860042070BD60
:20428000FF23EB4A7D33002808D0012812D0FF231E33022817D05F290EDB1BE0914201DD6B
:2042A00003207047994201DD02207047BE29FCDD012070475F2901DA002070479142EFDC22
:2042C0009942F1DC70475F29F6DB9942F0DB9142E6DC70479942EBDBFF20C3308142E3DB00
:2042E000DEE7F8B58026BF2704460D46002804D0012C08D0022C17D01FE0BE2D01DD012420
:2043000027E0002017E0FF207D30854201DD022410E05F2904DA0024204600F0E8FE0EE044
:20432000032000F0E4FE14E0FF201E30854201DA012402E0032000F0DAFE5F2D09DA694675
:204340000878C32130433840084001210C30084308E069460878C3213043384008400C30B3
:20436000400840000221084369460870009801F018FA2046F8BDF7B5AB4F82B0083FB8791A
:204380000D46002807D10120FDF793FC012001F0CAF90120B8710020FDF7A7FD04460120E4
:2043A000FDF7A3FD0090FEF7A8F839699E4E411A7D200001814203D29E48201804B233E03E
:2043C00038780099FFF75CFF387003283CD00020FEF746FD3878002838D0012839D00228D0
:2043E0003AD02821019178780099FFF77AFF7870CF2000F041FE022000F070FE072130689A
:2044000049058843052149054018306001F06AF8009000F06BFF019941180098081800B28D
:20442000211A0CB2FEF7D0FF20463B30772800D2002420464A30952810D2B87805280DD29E
:20444000401CB87000240BE00120C1E74B210901C8E7AF218900C5E78021C3E70020B87043
:204460003846FA787D230727DB007F061E2A02D20179322902D3012141712FE0002C13DA5C
:204480006D498C4201DC2B6009E0694963316118F92902D8FF21F53100E0FA212960521C54
:2044A000C2703068B84328E0002C17DD604A6432944202DB7D22920108E0FF3CF53CFA2C70
:2044C00002D27D22520101E07D221201491C2A60017130680121B84349060DE000212B6085
:2044E000C17001714279012A02D1544A2A60417130680321B8434906401830604A48FDF712
:20450000EDFC0220FEF766FF002801D0052500E003254B4C0020A07101212020FDF7F7FBFB
:2045200001212020FDF705FCA0790028FCD030680321B8434906401830603B48FDF7CEFCE8
:2045400004990020086002990874284605B0F0BD00230370AA23437010238370B423C37009
:20456000992303714C23437128238371FF23C371DD23037244234372F32383720B23037412
:2045800014201060294808600320704770B50646254814460D460722016852069143032256
:2045A000920689180160FDF799FC00233374236005202B6070BDB0B51921490186B0481037
:2045C000FDF785FB0520FDF78FFB0020FDF795FB1C4D80242846FDF797FB2846FDF7A6FB1C
:2045E0001949600101250860FDF7A0FFFDF77AFC0D49220308398860C008C000801C104352
:20460000072252050831104308600846FDF766FC0320694608741F2048748D74CD7404A84B
:20462000FDF7E1FB304611E0CC0C0020307500008A020000D8DCFFFF12FDFFFF50C3000048
:20464000981000209000030000E100E020434C21084302273843284300F00EFD022000F007
:204660003DFD042001F070F8042001F07AF800206946009008714C718C71CC710C724C72F1
:204680008C72CC72684600F0DCFE012000F098FF0020FEF7E5FB032000F029FD0321072045
:2046A00000F045FD0120FDF7B9FA6946087B8321204308400C302843384369460873039898
:2046C00001F06FF800F012FEFEF77EFE06B0B0BD1CB5FDF707FC454CA060FDF7FBFBE0606B
:2046E000FFF769FFFDF709FF0125414E2061FDF73AFF04463F480021CA00825CAA4208D19E
:20470000C9000818436801AA694639489847054603E0491C89B20529EED3307C00282CD0BE
:204720003348801CB06200207074B07431782F480C30417071788170FDF7C8FB307C2B4A69
:2047400001070832106800010009084307214906884301218906401810601046FDF7BEFB8C
:20476000FDF7CBFE0746FDF7C8FEC01BC82802D8B07C0128F7D10020B0740198FDF7CFFE15
:20478000FDF7F1FE071B0098FDF7F0FE8742F7D9ADE770B50446C1060120154D002900DAB1
:2047A000A874A1060AD512492031887100212020FDF7BFFA01212020FDF7A9FA200613D59D
:2047C000687C401C6874687C0B49C007A86A04D0421CAA620078487003E0421CAA62007879
:2047E00088700548FDF772FB70BD0000C40C002078100020FC5C0000D00C002030B5FE4ACD
:20480000002351780224142902D3537093702FE0F94DED1C48555078401CC1B25170012931
:204820001DD1D078202801D2032017E0802806D22038C5172D0F28180011001D0EE0E028B9
:2048400006D28038C5176D0F2818C0100A3005E0E038C517AD0F28188010163090701078F3
:20486000002801D0012804D19078814201D15370147030BDE04800787047DF48C078704703
:20488000DD48C01C70474178DB4838380170022070474178D8483838417003207047D648D8
:2048A0005838006C704770B5D34C0546583C206C401C2064FDF7C1FD216C022902D004294D
:2048C00003D006E000F0B6FA03E0CB4846211838C180FDF712FEE064C748012169563838E9
:2048E0008170084600F0B1FA00F0BDFA032070BD4178C1483838C170032070474178BE48EB
:204900003838017103207047BB49407838394871052801D3CD2801D9002070470220704775
:20492000B54918398A7A521CD2B28A720B795B1C0B714078FF2803D1022A01D34620C8805E
:204940000320704710B54178012909D18078002806D1A94818380079022801D8FDF764FDF2
:20496000032010BD032070470220704770B5417800220B06A0495839CB638A6384782504C9
:2049800094186B418C63CB63C5782D02A4186B418C63CB630579A4186B418C63CB634679EF
:2049A000350A3606A4196B418C63CB638679350C3604A4196B418C63CB63C679350E36023C
:2049C000A4196B418C63CB63007A20185341CB638863022070BD10B5874886B00024583825
:2049E00004705520FEF761F80220694608731620487301208873C87303A8FDF7F4F9FDF76C
:204A000071FA382188432830059005A8FDF766FA7A480168020611430160012000F0D0FD53
:204A20000020FEF71DFA764801690122520311430161734840308169090A0902091D8161B9
:204A400000F0AAFE69460490087C4006400E0874049800F0A6FE694600940C714C718C713D
:204A60000720C8710872684600F010FE0020FDF7B6FC0120FDF7D2F86420FDF750FD60489E
:204A800080380169FF2212029143192252028918016106B010BDF8B5FEF774F8FDF7C4FC14
:204AA00000F0A8F9544E4620183EF08000243546403DB47201272C645048AF700168020675
:204AC000114301602046FDF78AFCFF20F530FDF726FD0120FDF783FC0C20FDF720FDFEF720
:204AE00026F8FDF7E8FA002000F070F9FF214548F531FDF7F0FB6C703F48AF7044700470ED
:204B00003771FDF7FAFC68600120F8BDF8B5FEF7C6F8394D0746583D68780024364E0128EC
:204B20001ED0294640310620085EFEF748F8FDF7E4FC7D21C01BC900884217D8FDF7DDFC4A
:204B40006968401A782811D83078002815D0FDF7D4FCE860FDF7D1FCA860012068700CE032
:204B6000FDF7CBFCA968401A142802D96C700020F8BD30783346022801D00120F8BD6C7079
:204B80001C70D8780024204A2146CE00965D864206D1D81CC900891849688847044603E0D9
:204BA000491C89B20B29F0D3FDF7A7FC68612046F8BDF8B5FEF773F80F4C0746583C6078C2
:204BC00000260D4D012830D0214640310620085EFDF7F5FFFDF791FC7D21C01BC900884253
:204BE0002BD8A078012806D1FDF787FCE168401AC82822D8A67009E000110020801000F0E6
:204C0000005100F068360200245D00002878002819D0FDF772FCA061FDF76FFCE061FDF78A
:204C20006CFC2061012060700DE0FDF766FC2169401AFF21F531884202D966700020F8BDDD
:204C40002878022801D00220F8BD66702E70EB7800205A4A0146CF00D75D9F4205D1E81C42
:204C6000C90089184968884703E0491C89B20B29F1D36670F8BDF8B5FEF711F80746FEF757
:204C800014F8009000F0A9F84D4C0025607826465836012842D0214640310620085EFDF7C4
:204CA0008EFFFDF72AFC7D21C01BC900884206D8FDF723FC0099401A4249884204D9657056
:204CC000FDF786FC0020F8BDFDF717FCE16C401AFF212D3188420ED9206C02280BD9FDF71E
:204CE0000CFCE064012000F071F800F0BCF8FDF704FC20652EE0307800282BD0F078032865
:204D000002D0042804D006E0FDF7F7FBA06102E0FDF7F3FBE061012060701BE03078022831
:204D200018D165703570F2780020244B0146CF00DF5D974205D1F01CC900C91849688847E0
:204D400003E0491C89B20B29F1D365700328BAD0FDF73EFC0320F8BD194800787047FFF7C2
:204D60003AFE1420FDF7DBFBFF21F5311648FDF7B2FA134C2078012806D0022817D0032887
:204D800018D0FFF788FE01E0FFF7C0FE207000F01BFA0028EED10121102000F00EFD012030
:204DA00000F06AFC00F010FA0328FBD1E2E7FFF700FFEBE7FFF75FFFE8E70000245D000078
:204DC000A8100020AC0D000068360200974948718871704795480079704794484038006C8C
:204DE0007047924940390864704790484038808B00B27047F8B58D4C0025403CE56265638B
:204E0000256265620127A562FF202763F530E560A0616561FF202560C330A560E0612046F8
:204E20002030824E05763571FDF767FB20643572F771F8BD7D4810B5012120380176FDF724
:204E40005CFB7A494039C86310BD784A10B5403A11680B464143CC17640E6118CC1119199B
:204E60005161506010BDFEB5002668460671FDF71CFF02906D482038007E00287ED0FDF76F
:204E800007FF01287AD0FDF7D5FA012876D0FDF734FB664D403DE863FDF72FFBE96B401AFD
:204EA0000428F9D301E0FDF730F9FDF726FBE96B401A0628F7D35D4CA079012804D004205E
:204EC000FDF738F9FDF7E8FE0120FDF733F92860FDF7F1F80127277129686869401A009021
:204EE0006868C11C072908D200980F2801DD0F2025E001460E20C0431FE0014609311329E6
:204F000008D200981E2801DD1E2018E001461D20C04312E013302728009807D2322801DD11
:204F200032200CE001463120C04306E0502801DD502004E001464F20C043814200DA009022
:204F4000E8690099401800906079012802D06671A67128E0AF2100988900884202DD0020FB
:204F6000FDF7A0FEA07901281DD1E86932300090A671FFF794FC2E490A6800E054E09042C0
:204F800005D14868401C4860022809D200E04E60FDF7B3FA0299401A4B21C900884202D984
:204FA0000120FDF77FFE192000994001814203DCFF20A530814201DA009003E0FF209130C5
:204FC000814202DBE079002814D0FF2000999130814202DAE079012812D0207A002804D0BA
:204FE00068460079FCF727FF2672686800280DD000980DE01620694608712772E771EFE75A
:205000001220694608712772E671E9E7E8690090FDF7B6F9FFF743FC054908600098E86126
:20502000FDF76BFA28642671FEBD000058110020D80C0020F948816A490849008162816A18
:20504000022291438162816A042291438162816A082291438162816A102291438162816A22
:20506000202291438162816A402291438162816A8022914381627047E849C20703D08A6A77
:2050800001231A438A62820703D58A6A02231A438A62420703D58A6A04231A438A62020752
:2050A00003D58A6A08231A438A62C20603D58A6A10231A438A62820603D58A6A20231A43AC
:2050C0008A62420603D58A6A40231A438A62C00903D0886A8022104388627047CF498A6AF4
:2050E000FF231B049A43000402438A627047CB4AD16AC02380079943000E0143D1627047D4
:2051000070B5C74B81071A780025C44CC026090E904205D05A78042A02D2521C5A7070BD2C
:20512000E26AB2430A43E2625D70187070BD10B5BA4AD36A06248907A343490F0B43D3629A
:20514000D16A382340079943800E0143D16210BD08B5B24B403B5A6A0092012902D0002914
:2051600002D004E0024300E08243684602800098586208BD08B5A94B403B5A6A009201299C
:2051800002D0002903D006E0110C014301E0110C8143684641800098586208BD08B59F4B0B
:2051A000403B9A6A0092012902D0002904D008E01104090E014302E01104090E814368460D
:2051C00041700098986208BD9448806A0004000E704792498A6AFF231B029A430002024306
:2051E0008A62704710B58F4900F0EDFB7F21C90500F0E1FB00F099FC8849C0B2CA68120A47
:2052000012020243CA6010BD10B5CA07834CD20F030000F0F1FC09060C12181E242A303601
:205220003E00E0680121C9058843D1052FE0E068012189058843910529E0E068012149052E
:205240008843510523E0E06801210905884311051DE0E0680121C9048843D10417E0E068BE
:20526000012189048843910411E0E06801214904884351040BE0E068012109048843110415
:2052800005E0E068012212069043C907C9090843E06010BD61494039CA6B120C1204024308
:2052A000CA6370475D490A68120C120402430A6070475A494A68120C120402434A60704729
:2052C00056494A68000492B202434A60704710B5322100F0D9FA0006010A50484038C26B66
:2052E000FF231B049A431143C16310BD4B484038C06B32210002000E484370474749403967
:205300008A6AD200D208400702438A627047434A403A916A03239B06800799430009014345
:20532000916270473D484038806B0002000E70473A484038806B000E704738490A69027004
:205340000A691204120E42700A691202120E82700A69120EC2704A69027149690904090E98
:205360004171704730B52D490A6B0378120A12021A430A630B6BFF2212024478934324021C
:2053800023430B630C6B130285789C432D042C430C630C6BC5782402240A2D062C430C63A9
:2053A0004C6B0579240A24022C434C634C6B457994432D022C434C634C6B85799C432D04E8
:2053C0002C434C634C6BC5792402240A2D062C434C638C6B057A240A24022C438C638C6BF6
:2053E0009443427A120214438C638A6B9A43837A1B041A438A638A6BC07A1202120A000623
:2054000002438A6330BD00280ED0012810D0022812D0142010706E2011E00000405000F09F
:20542000E00C002000002041262010708A2006E004201070962002E01120107074201870A0
:20544000704730B552490A680378120A12021A430A600B68FF22120244789343240223436B
:205460000B600C68130285789C432D042C430C600C68C5782402240A2D062C430C604C6889
:205480000579240A24022C434C604C68457994432D022C434C604C6885799C432D042C435B
:2054A0004C604C68C5792402240A2D062C434C608C68057A240A24022C438C608C689443BF
:2054C000427A120214438C608A689A43837A1B041A438A608A68C07A1202120A00060243E0
:2054E0008A6030BD2A4810B58038C06B294900164843294900F0DEF900B210BDF8B5244DD2
:205500000E46303507460024A0000090C019401C00F0F6F901020098641C385C014302C563
:20552000032CF1DB00242D1DA700B819401C00F0E7F9F15D0002084301C5641C022CF3DB81
:20554000F8BD00B5C907124AC90F030000F054FB0504090E13181E00106A80239843C90170
:2055600012E0106A4023984389010DE0106A20239843490108E0106A04239843890003E058
:20558000106A0223984349000843106200BD0000805000F008520000FF0F000010B5FFF7EB
:2055A00013FE032807D00120C002B6490968884304D0002010BD01200003F6E7012010BD0A
:2055C00010B50446FFF700FE032808D00121C902AC4A012C106805D08843106010BD01213E
:2055E0000903F5E70843F8E7A6490A681202120A000602430A607047A2484068C0B27047E1
:20560000A0494A684006120A1202400E02434A6070479C494039CA68000492B20243CA603E
:20562000704798494039CA68120C12040243CA60704794498A691202120A03061A438A617C
:20564000CA690004120A1202000E0243CA6170478C4A403A91690223C0079943800F0143C9
:2056600091617047874940398A69C00752085200C00F02438A617047824A403A9169402379
:20568000C0079943400E0143916170470178CA014178890111438278D2000A43C178890076
:2056A0001143027952000A43D1B242790A4375494B691B0A1B0213434B618279C379D20131
:2056C000DB001343007ADAB210434A69FF231B029A43000202434A6170476A4940394862F2
:2056E0007047684A403A012905D0002902D1516A814351627047516A0143FAE761494039E0
:20570000886270475F4A403A012905D0002902D1916A814391627047916A0143FAE75948A0
:205720004038006A7047574A403A116901231B03C0079943C00C014311617047514840380C
:205740000069C004C00F70474E498A681201120F000110438A681202120A000602438A602E
:20576000704748498A68F123120E1A40400010438A681202120A000602438A607047414936
:205780004A691201120F000110434A691202120A000602434A6170473A4880690004000EC1
:2057A000704701B537498869FF22120290436A46127812021043886108BD324A0129916914
:2057C00008D0C043C0B201409069000A0002084390617047C9B20143F6E72A49FF23403999
:2057E0001B040128086B07D04002400E0A6B00049A4302430A6370470002000E80221043C3
:20580000F4E7204940390128886B07D0FD2210408A6B120A120202438A63704702221043E4
:20582000C0B2F5E730B5174B403B1C69FF252D04AC43000404431C6118690002000A09062B
:20584000084318615869000A000210435861986801210843986030BD0A4948690003000F43
:20586000C01C0F2800D30F204A691202120F120102434869FF231B049843120410434861F4
:2058800070470000405100F030B50B46014600202022012409E00D46D5409D4205D31D4661
:2058A0009540491B2546954040191546521E002DF1DC30BD70B500242546002801DA012488
:2058C0004042002901DA01254942FFF7DDFFAC4200D04042002C00D0494270BD03460B4334
:2058E0009B0703D009E008C9121F08C0042AFAD203E00B780370401C491C521EF9D27047FA
:205900000321001D401E037812021A43491EF9D510467047F8B502464A40D40F42004B00CB
:2059200052085B089A4202D20246084611464A0023D0C30D4A00DDB2120EAD1A202D35DAE4
:2059400049020126490AF6058A19002C00D0524220214F1B1146B9402A411018C20D9A421B
:2059600021D0002C17D0012D08DCDA05801AD20F8019D207DBB200F0F4F8F8BDDA05801AAE
:20598000012340001B06C01880185A428018CA0F1043490007E04908C2071143DA05801A9B
:2059A00080194008801800F0D4F8F8BD61000122511A001BF7E70122D2075140AAE70122D4
:2059C000D2075040A6E7024670B54A40D30FDB0740002DD04A002AD0010E140E000212024E
:2059E0000919400A520A8418E50104465443000A120A2E045043A4194219200CC543AA1883
:205A0000120C0125AD03521C521912047F39240400D0521C104301D44000491EC2B20C0630
:205A2000C0092018401C4008802A02D003E0002070BD40084000002900DA0020184370BDE2
:205A400070B502464A40D50F40004A00ED0740085208002814D0002A12D0C40DD30D41023F
:205A60000120C0055202490A520AE41A091812187D34914201D3641C00E04900002C01DAEC
:205A8000002070BD0023914201D3891A0343400849000028F7D100290AD0914202D10121BA
:205AA000C90705E0914201D2012101E00121C943E005C018401900F04CF870BD420005D0CC
:205AC0004200120E52428A4201DB00207047C90508187047C217C10F504010B54018CA0785
:205AE0009623002100F03DF810BD10B500229623114600F036F810BDC20F41004002012380
:205B0000400ADB05D207090EC0187F2901DA00207047962903DC9623591AC84001E09639B7
:205B20008840002AF4D040427047410040020122400AD205090E80187F2901DA00207047A6
:205B4000962903DC9622511AC8407047963988407047002904DA401C490001D14008400071
:205B6000704770B40024050C05D11024000402D1002921D01124050E01D100020834050FAE
:205B800001D10001241D850F01D18000A41C002801DB4000641C002908D020252E1B0D46A5
:205BA000F540A14000D001212943084301061B1B000ADB1D02D5002070BC7047DB051818FD
:205BC00080180029F8DA401C4900F5D170BC400840007047064C0125064E05E0E36807CC8D
:205BE0002B430C3C98471034B442F7D3FBF722FB7C5D00009C5D000030B47446641E25786E
:205C0000641CAB4200D21D46635D5B00E31830BC184702E008C8121F08C1002AFAD1704729
:205C20007047002001E001C1121F002AFBD170470101000100000101000001010000010103
:205C4000000001000100010100000100010100000100010001000101000001000101000134
:205C60000001000001010001000100010000010001000000010000003934000002000000AC
:205C80006F34000003000000CF350000040000006D390000050000005B3A00000600000010
:205CA000793A0000070000008D3A0000090000009F3A000020000000AF3A00002200000056
:205CC000E93A000028000000FD3A000031000000D13B000051000000E73B0000540000003E
:205CE0000D3C000055000000293C000071000000453C000081000000853C0000010000006C
:205D000025420000020000005142000003000000774300000400000051450000050000002B
:205D20008D4500000100000087480000020000009348000003000000A748000004000000EE
:205D4000F148000005000000FD4800000600000009490000180000002149000028000000BE
:205D60004549000051000000654900007100000069490000810000006D4900009C5D000043
:205D8000800C002064000000125C0000005E0000E40C002080040000225C00000000000015
:205DA0000000000000000000000000000000000000000000000000000000000000000000E3
:205DC0000000000000000000000000000000000000000000000000000000000000000000C3
:205DE0000000000000000000000000000000000000000000000000000000000000000000A3
:00000001FF
